:1000000002037BEFD394077480948040037FFF2228
:100010001202D3FED394037480948040037FFF22A6
:10002000EF7044EE700B9000011202ECF452935208
:10003000941202D36401700B9000011202EC4293FF
:10004000F452941202D3FE6402700A90000112026C
:10005000EC42934294EE6403700D9000011202ECA6
:10006000FEF45293EE4294EF640170461202D3FE06
:10007000700B9000011202ECF452915292EE640166
:10008000700B9000011202EC4291F452921202D3D2
:100090006402700A9000011202EC42914292120234
:1000A000D36403700D9000011202ECFEF45291EE45
:1000B0004292EF640270461202D3FE700B90000170
:1000C0001202ECF452955296EE6401700B9000010E
:1000D0001202EC4295F452961202D36402700A9016
:1000E00000011202EC429542961202D36403700D95
:1000F0009000011202ECFEF45295EE4296EF64037A
:1001000070461202D3FE700B9000011202ECF45202
:10011000B152B2EE6401700B9000011202EC42B1D8
:10012000F452B21202D36402700A9000011202EC7F
:1001300042B142B21202D36403700D900001120268
:10014000ECFEF452B1EE42B2EF640470461202D3F8
:10015000FE700B9000011202ECF452B352B4EE6444
:1001600001700B9000011202EC42B3F452B412027F
:10017000D36402700A9000011202EC42B342B4123E
:1001800002D36403700D9000011202ECFEF452B32E
:10019000EE42B4EF640570461202D3FE700B90007D
:1001A000011202ECF452C952CAEE6401700B9000C5
:1001B000011202EC42C9F452CA1202D36402700A5C
:1001C0009000011202EC42C942CA1202D3640370C9
:1001D0000D9000011202ECFEF452C9EE42CAEF6427
:1001E0000670461202D3FE700B9000011202ECF46E
:1001F00052CB52CCEE6401700B9000011202EC4223
:10020000CBF452CC1202D36402700A9000011202A5
:10021000EC42CB42CC1202D36403700D9000011269
:1002200002ECFEF452CBEE42CCEF640770491202AE
:10023000D3FF7E00700B9000011202ECF452E152E9
:10024000E2EF64014E700B9000011202EC42E1F407
:1002500052E21202D36402700A9000011202EC42D0
:10026000E142E21202D36403700D9000011202EC2D
:10027000FFF452E1EF42E27F002212036BC2C87F1B
:10028000C87E00120343D2C87FC87E00120343C257
:10029000C87FC87E00120343D2C87FC87E00120305
:1002A0004312035A7F017E00120343D3E5089405ED
:1002B000748094805003120387050AE50A700205D2
:1002C00009C394E8E509940340DAE4F509F50A0561
:1002D0000880D1BB010689828A83E0225002E7228E
:1002E000BBFE02E32289828A83E49322BB010CE5F0
:1002F0008229F582E5833AF583E0225006E92582DA
:10030000F8E622BBFE06E92582F8E222E58229F51D
:1003100082E5833AF583E493221202D364017003E9
:1003200075C1209000021202EC5407FFE5C154F899
:100330004FF5C19000011202EC700453C1F7224343
:10034000C108227D607C09ED1D70011C144C70F702
:10035000EF1F70011E144E70EA22750B01E4F50CBC
:10036000750D03FB7A00790B020319750C01E4F596
:100370000BFB7A00790B7F05020003787FE4F6D847
:0B038000FD75810D02027A43C11022BE
:00000001FF
